:100000000C940D130C94E0160C94FC160C942A130B
:100010000C942A130C942A130C942A130C942A136C
:100020000C942A130C942A130C942A130C94831402
:100030000C942A130C942A130C9492140C942A13E3
:100040000C942A130C942A130C942A130C942A133C
:100050000C942A130C942A130C942A130C942A132C
:100060000C942A130C942A131E00000000000000B8
:100070000008820042000000100806830100000012
:1000800000020000840EDD79180004060C000088D0
:10009000114200003C0000000000000000000000D1
:1000A0000000020000F8000000BEC576790E0000D6
:1000B0000000000000000000FF0F000008314210A7
:1000C000080C0000FFD77FFF0F0000100000048124
:1000D0000030303019FF00048100001C8E4C0000FD
:1000E0000602000000BE81F16AA5566A0538040CBC
:1000F00000000C00A1C43052C830F3CC3080274936
:100100001E00000C03007F1886E1FFFFFFFFFF00C9
:1001100000000000000000008550A0101A020C032F
:1001200084A1C4305208000000001E000023490CC6
:1001300000000C03005E1886A1073092C40000C0C6
:100140003000F0FFFFFF03FFFFFFC0FFFFC0FFFF16
:10015000FFFF03FFFF03FFFFFF6AA5566A55A9953E
:100160005AA92084104200E39C730C38EF7FCF0122
:10017000FB9EF70D4F1086207F866118E26318867C
:10018000611CC6613886609C966300C26939042090
:100190008C164300C208310420841042004008211C
:1001A0000000801000E08561187A0023490C0000EF
:1001B0000C03000007002DF0FF400BFC00F00312C1
:1001C000D0B68034CF0C33CF00000000104A042298
:1001D0008500000000001E0001000000300C00003F
:1001E00000857100009028CC03009144611F108AA3
:1001F000240AFF8040201008000402810000201023
:100200000800000081000000000802000000300C1F
:100210000000806238000024C5F000204A8AE10313
:10022000619414C30F4008210400801042000000B4
:1002300021040000004200000000040C000000E067
:1002400031000000BFC70000D0FE1E03004CFB7B46
:100250000CC030EDEF314CC8844C18322113320001
:100260001E0041108620280892044104C130080273
:100270002194420800E0790020100A854008C2302D
:10028000040141922408201886410084611802412B
:10029000108620280892044104C1300802219442AB
:1002A0000800E0790020100A854008C230040141AE
:1002B000922408201886410084611802411086208B
:1002C000280892044104C13008022194420800E049
:1002D000790020100A854008C230040141922408A8
:1002E0002018864100846118020018007FD8B6A348
:1002F000FF876D4BFE7FD8B2E9FF876C1BFF3FD8AD
:10030000F6E1EF877D1BFE7DDCB6E1BFA76D1BFE2E
:1003100077D9B6E1FF8E6D1BFE5FF8B6E1FF07ED02
:100320001BFE7FD8B4E3FF876D53FE7FD8B6C9FFAD
:10033000876D1B7F7FD8F6E1FB877D1BDE7FDCB6F8
:10034000E1FEA76D1BF67FD9B6A1FF8F6D1AFE7F68
:1003500078B6E1FF85ED1BFE1E00000000520B0089
:1003600080D4020020B50000482D0002520B00107E
:10037000F003008000AD04000400B412200000D09F
:100380004A010004402B01800000AD04100000FC75
:10039000000200520B4080D4020028B50000482D16
:1003A0000002520B0010F003008000AD04000400B6
:1003B000B412200000D04A010004402B018000004C
:1003C000AD04100000FC000200520B4080D402007B
:1003D00028B5000000FF0F0000F3FF0CC030FFCF76
:1003E000300058002008822008C3300CC3388661D2
:1003F00018CE330CC3F0BE611886FF0FC330FC7FEC
:100400001004C1FF030000FC3F0882E0FFC3300C72
:10041000FF1F8661D8F7B22CCBBEB76DDBF6BD6D82
:10042000DBB66D6DD3B46D6B1BA66DDBFB30EFDB04
:10043000DE0779DFF43EC0FB86FF03FE3FFC3FF0A2
:10044000FFC1FF03FF0FFC3FF8FFC0FFC3FF07FC26
:100450001FF63DC0F7B2EF09BEB77DCFF0BD6F5BB1
:1004600086ED7DD3304CEF1B8661F8FF300CC3FF67
:10047000074110FC3F0000C0FF832008FE3F0CC373
:10048000F0FF6118867D2FCBB2EC7BDBB66DDFDB36
:10049000BE6FDBDEF47DD3F486EF1B863FFCFF30BE
:1004A000FCC1FF07C10FFE3F00FCF0FF83E08F7F20
:1004B0001F0CFFDCF360D8E79E27CBBCF73CDBC604
:1004C000BD6599266C2DCBB6616BDBB60DDBFBB63B
:1004D000EFD8DE377DCFF4BEE1FB86FF0FFF3FFC98
:1004E0007FF0FFC1FF03FF0FFC3FF0FFE0FF01DFE4
:1004F0000FFF0FF07CD87782E7CBBE333CDFF69D51
:1005000061D9B6ED0CC3344D6F188661F8C3300C59
:10051000C31F044110FC000000C00F822008FE3001
:100520000CC3F08F6118867D0CC330CC6B188661CC
:10053000DCC3300CC31E044110F4200882A00FC39A
:10054000300CFF188661D8CF300CC3FC866118C60A
:100550003F0CC330FC411004C1070000003C000008
:1005600000C0010000000C0000004000000000007E
:100570000800000800010042602004100209848085
:1005800010088110844020102204020442011080CF
:100590000008006000002D00000000400000000086
:1005A0000800000000010000002800000000050015
:1005B0000000A000000020040000088000000220CD
:1005C00000800008002000020000810000002800D8
:1005D000000040010000000A000000500000000080
:1005E0004200000010000100004000040000000173
:1005F00010000000040200000040000000000A009B
:10060000000040010000400800001000010004400C
:10061000000020100000000500000028000000007D
:1006200021000000088000000020100000000003EE
:10063000000080200000000C0000004000000008C6
:1006400000000001400000000C000000011000004C
:100650000004400000001000010000400004000001
:100660000000000016000000000000020000001062
:1006700008000080402000000402810020100804CF
:10068000028140201008040281400010080402008A
:1006900040201000000081000000000400000081E4
:1006A0000000402010001008040204028140814034
:1006B000201028100804020402810080402000005D
:1006C0001008000000000000000011000000000001
:1006D00010020000848004001200000C030080C49B
:1006E0003012104A0C238500C03000004800200161
:1006F00000C0300000789EE701FFFFFFFF0F7892F7
:10070000E40100C03000F0FFF3FCFF7FD8B6E10F3A
:100710007892E40100000000000005002100004084
:10072000080500000A08108000410060002002084F
:100730000001040014000000004000000020000040
:10074000001000000008000000040000000200008B
:1007500000000800000000200000000080000000F1
:10076000000002000000000800000001000020005E
:1007700000000400008000000010000000004000A5
:100780000000000001000000000400000000100054
:100790001E0020060946C03000C0308121401808E4
:1007A0000008010000402000000008010000402077
:1007B00000000000000C000000800100000030007C
:1007C00000000006000000C0000000200800000833
:1007D00002000082000080200000200800000003CA
:1007E00000000018000000C000000000060000002B
:1007F0003000000000410000000004010000001073
:100800000400000040100000000041F0FFFFFFFF67
:10081000000000000000000000000A004110044138
:10082000200882200804411004812008822010043E
:100830004110048220088210044110842008822084
:100840000441100421088220080006002084104280
:100850000021084108024120081408040281406078
:1008600060200080981100001A0000000040000085
:100870000020000000040000000200004000000012
:100880002000000000000100000000020000000045
:1008900010000000002000000000000100008000A7
:1008A00000001000000008000000010000800000AF
:1008B00000000004000000000800000000400000EC
:1008C0000000800000000000040000000200004062
:1008D00000000020000000040000000200000000F2
:1008E0000100FFFFFFFF0F00220000C03000007872
:1008F00092E4017F1886E13F870010CE0C1086003D
:100900000360906000802140180000080100004052
:100910002000000008010000402000C0486128318C
:100920000023490C30870010CE80C4301200309272
:10093000C40000C03000104A002085502240A4208E
:100940009090904000E27004104A002085502240B0
:10095000A42090909040710000E0881091881000D1
:10096000462606408900102980C43012003092C407
:1009700000A1040052E88561187A8027491E100200
:100980000C0384000C0028A5504A51289442A12051
:10099000A5564A40A99158296A05006A55A90050F0
:1009A000A96A55A96A05A86A55014055A92AA0AAAD
:1009B0006A55555555A9AA7AE0077EE01F002D100B
:1009C00086402B8500104A0023490C00000C0300D0
:1009D00021000040084800200100C0300000309293
:1009E000C4000C10860033820412C4589090A06199
:1009F00080641260718010E0C800650A302388109E
:100A0000418C05050A1A06881601160704028E0C89
:100A100090960023850C134A0023490C60806010D7
:100A2000608007001E00846118021E0000800750CD
:100A300094A20080A250140014058A02008A1605B0
:100A40008001030C1861080061089000C2000000DA
:100A5000201C060000C2E13000201C0E8701C2E10C
:100A600070380C100E87C3008070380C000084C3EF
:100A7000000040BB0C008071CA00C0388700609C39
:100A8000730830CE398700E39C430030CE2100004C
:100A9000E31000433008603804000C874380E170A5
:100AA00038341C0E8743C3E17008301C0E0100D39C
:100AB0002D000030E518000010CE310000E19C63ED
:100AC0000010CE39C700209C730C004038C700C10D
:100AD00084730C100C08C700E198700C10CE31C163
:100AE00000E19C630000C239C7000084730CC2009F
:100AF00008C7201C06100CC2E13000201C0E870124
:100B0000C2E170380C180E87C380C070380C08041E
:100B100086C3804020303C0C0402C386412018C6A6
:100B2000300CC3301886108601C308310C008C1FAE
:100B3000030000FB0D000070EF00000C070E03C364
:100B40004020300C0C070E030070EF000000FB0D7E
:100B500000008C1F0300C308310C008C1F03000031
:100B6000FB0D000070EF00000C070E03C3402030A7
:100B70006C180482610C43200CC33008C130188605
:100B8000108601C308310C18861086C13008C130A8
:100B90000C43200C6318048261C34020306C18049D
:100BA00082610C43200CC33008C1301886108601C6
:100BB000C308310C008C1F030000FB0D00C070E067
:100BC00030300C0402C386412018C63004C23018ED
:100BD00086108601C308310C008C1F030000FB0D3A
:100BE00000C070E030300C0402C386412018C630CB
:100BF00004C2301886108601C308310C008C1F0314
:100C00000000FB0D0000A0590020089A054182A4B5
:100C1000591224499A254992E47992F4030C03FC71
:100C200061D8B66108FC0CF303D2EF79BF24FD92C2
:100C3000F44BD22F49BF24F992E44B122F49BC2424
:100C4000E192844B122C49B0248192044A1220492B
:100C50008004009E070000E3790CC030FFCF300C09
:100C600033CF0CC30061083000C0300000309EC795
:100C7000000CF3FF0CC330F3CC300C1086000300E3
:100C80000C03000023490CC030F3CC300C1086005C
:100C900003000C030000E079000000FF0F0000F0EB
:100CA000FF000300DFC73000F03C0C0300C7C33077
:100CB00000F33C0CC3304DC3300CC3300CC0300CBF
:100CC00000000C030000C000000000000000000055
:100CD0000000000019000040200000080000010191
:100CE00000000008040108020008060100030000DB
:100CF0000C0C00000033000000C040108020008079
:100D00006010002004004200000C030080C4301278
:100D1000104A0C23850023490CE0B5F3DC7A5E3BD6
:100D2000CFADC778F3EC3180C43012007892E40183
:100D300000C0300000480C2301A1C4305208480014
:100D4000200100C03000000027007F1886E10F005E
:100D50000C03007F1886E10F000C03007F1886E16A
:100D60000F000C03000023490CC030F3CC3000C04E
:100D70003000003092C4000C33CF0CD3026D0BB4A2
:100D80007FD8B6E1DFB6FFDFB661FBFF6D1886FFE7
:100D90001F866138CF611886611886611886611BCD
:100DA0008661D8FE6118B67F1886ED1F8661FB87C5
:100DB00061D8FE611886ED1F86E1DFFE61F8B7EDB0
:100DC0001F867F1BB6FFDF8641FBFF2D1834FFCF48
:100DD0008240F3FF2C0030FFCF0000E37F0C003097
:100DE0009EC700FF1C86F30F309EC700FF1C86F3D2
:100DF0000F309EC700FF1C86F30F23008C14861251
:100E0000C348652A318CD4B61223B592D44AA104C2
:100E10000052288500104A520800A1A48500105AEB
:100E20005A0800A1A59500905A5A0900A9A5950055
:100E3000905A5A2940A9A59502945A5A2940A9A521
:100E40009562945A5A2946A9A59562945A5A2946F8
:100E5000A995916294885A2946A195916290985AD1
:100E60002944A995914294985A2146A99590629453
:100E700098522946A9C589639C395A0946A9959172
:100E80002294985A2946A8C599639C3918294689FD
:100E900001609C630000841002001E00010000003D
:100EA000080400000202000000440000002080004E
:100EB000001000000108000100090008280040019E
:100EC00004402000023000C00000C0300000480094
:100ED000200121000040E8856D1B7A5ED8B6A1177D
:100EE0007A92E485A127495EE8856D1B7A5ED8B6C3
:100EF000A107D102B4080027490E103096C6802001
:100F0000A3594C103896C68120A7594E10F992F477
:100F100089E227497E243C92C443C2214038240CF4
:100F2000000043002A001E00008027100A85401E92
:100F300000008027100A854000E0790080100284BC
:100F40001000E0790080100284101E000080E7018C
:100F500000007802A1500824100A854000E07900C2
:100F600000009E07000821400881100284109400B0
:100F70000090020902040908040902C1400020305F
:100F80000EC03000777892E4E143C030201C7C939F
:100F9000EC8340D0B62000F8F3FC0120C8364100B5
:100FA000FB92F40DA02F4F5F00F8F3FC01C037CF88
:100FB0003E007C97EE03C0E7793E00719EE708147F
:100FC000C5398A40519CA3081445208A425104A285
:100FD00028148110884211088128040400020202AA
:100FE000000004003A00FFFFFFFFFFFFFFFF7FFF4D
:100FF000FFFFFFF7FFFFFF3DFFFFFFDFF3FFFFF7FF
:101000001CFFFF7FCFF1FFDF730CFFF71C43F87F5E
:10101000CF3184DF730C21FC3DC710C2CF31843047
:10102000FE1C4308E3C710C2387F0C218CF3430831
:10103000E3BC3F8430CEFB218CF3FE1FC238EFFFB0
:1010400030CEFBFF0FE3BCFFFF38EFFFFF8FF3FE57
:10105000FFFFBCFFFFFFCFFBFFFFFFFEFFFFFFEF28
:10106000FFFFFFFFFFFFFFFFFFFFFFFFFFFFFFFF90
:10107000BFFFFFFFFFFBFFFFFF3EFFFFFFEFF3FFA1
:10108000FFFB3CFEFFBFCFE3FFEFF338FCFF3E8FDB
:10109000C3BFCFE370F8FB3C0E873E8FC3E1E0F3A4
:1010A000381C0E3C0E87C3C1E370381C381C0EC7B9
:1010B00083C3E1703C70381CCF0787C3F17CE170BB
:1010C0003CDF3F1ECFF7FFC7F3FDFF7F3CDFFFFF95
:1010D000CFF7FFFFFF7CFFFFFFDFFFFFFFFFFDFFFD
:1010E000FFFFFFFFFFFFFFFFFFFFFF0046002000A5
:1010F00000400082001004200806410082611804AC
:10110000601886611086611886631886613C8E615E
:1011100018C7E338C6713C8EF31CC7E33CCF733C61
:10112000CFF33CCFFB3CCFF3BDEFF37CDFFBBEDF67
:10113000F7BDEFFF7FDFFBFFFFFFFDFFFFFFFFDFDF
:10114000FFFFBFFFFCFFFFF3C7FFFF3F3EFCFFFFBA
:10115000C3C1FFFF3F08FCFFFF0380FFFF1F00F03C
:10116000FFFF0000FEFF0700C0FF3F0000F8FF0187
:101170000000FF0F0000F0F90000000F0F000070EA
:10118000E0000000030C0000108000000061080077
:10119000001886010082611804301886C1808361BE
:1011A000181C3C1886C1E38361187C3F1886C1FF78
:1011B000876118FEFF1886F1FF9F6198FFFF1B866D
:1011C000FDFFFF61F8FFFF1F8FFFFFFFF3FCFFFF35
:1011D0007FEFFFFFFFFFFFFFFEFFFFFFE7FBFFFFCC
:1011E0007DBEEF7FDFE7FB9EF77DBEE779DEE77927
:1011F0009EE7798EE7791EE7389EC7718EE3701CF3
:10120000E7380CC3710EC3300CC7300CC33008C3B1
:10121000300C81200C431008821004812000401003
:10122000080000000100000000002B00A504065289
:101230000A3592C40A08D1B908514A6020A5502342
:1012400049AC40486C232184C4361252486821A11D
:1012500040A5562A0040FD2B00105AA9850042F5F2
:101260002A041052A98480109D8B108450A910224A
:1012700004970E428550A9100A14978E0280D4B6A6
:101280001220B500D04A1223498CC4300CC3308CD4
:10129000C43012238592144A522249A4A4140A8508
:1012A00052C660603006A0905000280E0947814267
:1012B0006A2514905AA99540AB99592D38BDD0CBC9
:1012C000816766661E994A2F9569560BAD66994AE5
:1012D0002F9599A9F452991C73E68C03AD15B24D64
:1012E00043C22D3739104BC2A3C0F0201804570059
:1012F0002084104200419020080804060201E0000A
:1013000070000012890400200C43000042290400F0
:101310003800C001082140084110048220028110D9
:1013200008043800C0018040201000089204010029
:1013300042290400009C030000A1500800200C4337
:10134000000084100200009C0300040209048220B3
:1013500008411010422084007000E00004020904DB
:10136000822008411008040602810300001C000EC0
:1013700000070000F801000070E000001C0080037E
:10138000070000001E080402814110802028080286
:101390000441044120088220084110100409820001
:1013A00082601004300C0FC380E3F8711C3CCF3F07
:1013B000CFE3FBFEF77DFFFFFFFFFF7D9FEFFBCF3E
:1013C000F3F03C7F1C078EE3C330C0301C040108DF
:1013D000828140201078000000E0C70100387E1CA8
:1013E000078EE3388E1FC701E0FF7F00C0F1FF3892
:1013F000701C078EE38EE3701CC7719CE338388E37
:101400001FC701E0FF7F00C0F1FF3800389EC70111
:1014100000E7790E00000C030000E3790CC030FFF8
:10142000CF300C33CF0CC300610830581080A011AE
:101430000700008E230800416C806010600C10864D
:1014400000830501081A710000E01802000084A161
:10145000040052184A0C2385C00F4892C4486128E2
:10146000319224013F104A0C238580C430120000C1
:101470000C030000000000006D007F1004C1FF0B92
:101480008220FC3F4110C4FF330CC3FC000000006D
:10149000F0330CC3FC3FC330CC0F000000003FC34F
:1014A00030CC0F00000000611886E11C866138878F
:1014B0006118CE611886611B866118B67318866143
:1014C0005A8F6118AEF7188EE37A8FE338AEF708BB
:1014D00000000000E338AEF7388EE37A8F0000009A
:1014E00000308EE37A8F000000001086610878617A
:1014F00018861E1086E10F0061F8870010867F288D
:101500000161F8871233867F2831E3F88712338E22
:10151000FF283100000000308EFF2831E3F88F12E1
:101520000300000000E3F88F1203000000000C101D
:101530000400033082C0000C330C0CC30CC33030E9
:10154000CF300CC3F30FC330FCFFBC0FC3FFCFFB86
:1015500030FC00000000F0CFFB30FCFFBC0FC30FDD
:1015600000000000FFBC0FC30F000000003F0000A0
:10157000C0FF0300F0FF3F00FCC0FF07C11FFC7F5E
:10158000107CC1FF0FC333FC00000000F00FC33319
:10159000FCFF303CC30F00000000FF303CC30F00D5
:1015A0000000006118866118C6613886619C9663E8
:1015B00038CEEB39860000000030CEEB3986E3BC34
:1015C0009E630800000000619C966318FE61F88726
:1015D000FF1F86FFFF876118FEFF3CCFF3FFCFF3AD
:1015E0003CFF00000000F0CFF33CFFFF3CCFF30FC7
:1015F00000000000FF3CCFF3EFCFF33CFBFD3CCFFE
:1016000073BFCFF33CEFF73CCFF3FD0EC330BCDF2D
:10161000344DD3F74CF33C3D00000000F04CF33C5C
:101620003DCF34CFD30300000000CF34CFD3F34DF0
:10163000D3347DFF340CD3FF0FC330FCFF301CC309
:10164000FF0FC333FC00000000F00FC333FCFF307A
:101650003CC30F00000000FF303CC3FF0FC333FC4E
:1016600000000000000028008000000000080000CA
:1016700000422100002014020000055208008020D2
:10168000C8010010042107008220841C0000801083
:1016900002000000420000000008000000000000FE
:1016A000000000000002000000200000000885008B
:1016B00000805008002094482100278A22C78941D1
:1016C00010886200004010000000000000000000D0
:1016D00000000000000004000000400000001008AE
:1016E00001000081100040201042000C044108035A
:1016F00081200841201006210804A22004810885C9
:101700008020805008002094482100278A22C78921
:101710004110886200004010000000002400010415
:10172000000200240000080411000000184000001E
:1017300040400001000000010604000014001000F9
:10174000801010400004004000210000000105004E
:10175000800004102004001000A0000040040102DA
:101760000000180008004040002000000009800828
:1017700000400400200002100280100000088002D7
:10178000000020040800008000A001000002040402
:1017900000002820100000018040000800000241E5
:1017A00000020008041400002080100000800640A1
:1017B00000002008000100012000040080800010CB
:1017C0000C008027491E007892E4018027491E8082
:1017D0005891A8118027491E007892E4018027497A
:1017E0001E40686264218027491E007892E40180CF
:1017F00027491E20B092D440080000C030000030BD
:101800000CC3000CC3300C03300CC30000C030000C
:1018100000009E070000F0FF0000009E07000C0083
:1018200030CE39C700E0FC730000EC7F030000FFFE
:101830000F00C0F0F930001C0F8F03C3E170386C4B
:10184000180E876186C3301CC6300CC33018C730F1
:101850008E81619C63183C00000010C6000000C22D
:1018600018008000180300040461000051000C40BF
:1018700010028200868020003024080080091200B7
:10188000008A02020030A0080080018420000C00C1
:101890001006600000C20003800018100404040158
:1018A0004010510000405102000086040100300445
:1018B0001004800110C0000802021800A0080003F4
:1018C00000842060000010060C0000C282008080AE
:1018D000380000240C010008530000C21002003040
:1018E00086000080310400008C01100060080202B4
:1018F0000003A0080010048420004010100600001F
:1019000041C200008004190000041405000051C009
:1019100000401002180086000003300400608001BF
:1019200010000C0802028200A088200000A42800F9
:1019300000081206008200C20030800018800104F6
:1019400004010C00510060401002000386000010EA
:1019500034040000C0111000000843020000A00C75
:101960000100008430041400800700C00F780010CC
:101970007C800704C1033843101CC0310CC1100C1B
:10198000C3300443300C077004C1E0004F10001E48
:10199000F0050CE3013FC0301EE0830CE3013CC8BE
:1019A000721C80833C8F0130CCF33000E23C0F820C
:1019B00000CFB3200C782C0BE280C7B0200F780C3E
:1019C00003F81A00330300CC0C000C0300330300AF
:1019D000CC0C866118063F0000C0FF0B0402FDBF5F
:1019E0004820D1FF4B0C23FDA12449520842200876
:1019F00081AD0400001008412004000000523B8724
:101A00000010CE0CF3FF0C33870010CEF3CC30F374
:101A1000CC30F3CC30F30C00F30C000C0300C3C04B
:101A200030300CC30C330CF3CC30F3CC30F3CC306F
:101A3000F3CC30F30C000000000006002100004051
:101A4000288500104A8C148612C330F3CC3052EB38
:101A500079AD144A0C2385000900522B49AD24B5F9
:101A600092D44A522B49AD24B592D44A8CD4B612A2
:101A7000C3486D2B318CD4B612C3486D2B318CD436
:101A8000B61203002B002084104200A194520808D3
:101A900021460841080108214200002014000000EE
:101AA00080010000001800000080010000002804F0
:101AB000000042841080108210628410104A298530
:101AC000004208210420841042004208210420041E
:101AD00000420042002004200400420002000004F2
:101AE00020000040000200000410080081804060D7
:101AF000201004128904120804028142A1502844D3
:101B000020914820080406020181001008200000EE
:101B100040000200000420000040000200000420F9
:101B200000004000020000042000004000420020AD
:101B3000042004004200420020042084104200429D
:101B40000821042084104200280000C03000004812
:101B50000C230180D4B612107A6D2B85A1D77A524E
:101B6000184AAD37B7A1F47B731B4ABF34B7BFF433
:101B70004B73FB4BFF34B7BFF4CF73FB4FFF3CB746
:101B8000FFFCCF73FBDFFF3CB7FFFFCF730B000001
:101B9000C3489224318C244952DB4AD22FB5AD344C
:101BA000FF52DBCEF32CB5EDCC30AD24310C134A13
:101BB00012C300A124312D104A12D302A134B72D33
:101BC000307B73FB33AD27CDC02C852D33CF52D85E
:101BD000320CD37AD2EC79BF27CD6108842DD3861D
:101BE000DEDF32921702D22C79F3ECFD6DC8302182
:101BF000F0CF9E377B0013864C083061C8FC37005D
:101C0000311E21322AE31A8D0234CEF30080F33CD8
:101C10000E003C8FE300C0F3380E003C8EE300C0A2
:101C2000F3380E0038CFE30080E33C0F00388EF32A
:101C30000480E3384E10388EE30081E3380E000054
:101C40000EE0008003380000000EE0008003380042
:101C500000000EE0008003380000000EE00080036A
:101C6000380000000EE0008003380000000EE000A5
:101C7000800338000038C0010080030E0000387077
:101C80000000800303000038100000800300000003
:101C9000300200000042080000000821000000207F
:101CA0008400000080100200004042000008080884
:101CB00000010101003020000004050000C01000F8
:101CC000001004010000C1000000700000000007C7
:101CD00000000070000000008003000000001C00F5
:101CE000000000E000000000000300000000080009
:101CF00000000000000000000900000000000000DB
:101D000000020000002000000000000000000000B1
:101D10000000000200000000000000000200FFFFC1
:101D2000DFFF0F001A0000000000000000000000AC
:101D30008230000000000000008230000020080314
:101D40000000000000002008030000000000002048
:101D50000803000048210000801402000080E00019
:101D60000000080E00000021100800100281000091
:101D70006008020000862000002094000000420954
:101D80000000380800008083008040200400080420
:101D90004200008230000020080300001400288A5E
:101DA0001F4581A26F5F14E8DBB67DF1B66DDBF6EF
:101DB0007FDBB6EDFFB792D4FEEDEC79731BFEF33B
:101DC000FC87403BCF2DE0B5F3DC7A1E23498CE73E
:101DD000B5F3DC7A21D0B640184A6D2B858154A624
:101DE00012084A9A250581442012087A08E10581E3
:101DF00047201EC84A0821351A000000300C030095
:101E00000023850000FC0000003F0000A1C400008A
:101E100010862100008C14020000003F000000101A
:101E20004A0C000061180200C04821000000F003C5
:101E300000008412F30300C330C00F305208FCC00E
:101E40000F00A1C4FC00C030CC0F008C14FE0000B9
:101E500000FF0F0000F0033F00003F00FC00F00314
:101E6000520B00BFD40280D44A2D2014520BA10083
:101E7000270004C13F0842103CA32404C1330C4393
:101E8000103C439104C1F30441520C4F100CC3F0B9
:101E90000491280C4F1008F2F00491280C43910C87
:101EA000C3300C43520CA32408F2F004114A0C2353
:101EB0008504C13F08C250E483200CC33C08C230F3
:101EC000CC09210CC3FC00C0304C2E100CC3F00414
:101ED000C128094F100874E6020100FF0F0084902A
:101EE0009F101204F909824131C62818140D8B8203
:101EF0004152A9244828954A218412891402388A1B
:101F0000E200C051501C001C058A0300F0F60010CE
:101F1000086C038104C1360842120C83240CC130C2
:101F20000803250021000040080500000A08108071
:101F300000410060002002080001140200008450EB
:101F40000000A0800001081004000600228000109C
:101F500040210000400848002001002240040010F9
:101F60009080008004001200200244000001090853
:101F700000480020010001090800200244008004FC
:101F80000012001090800000224004004800200150
:101F90000001090800200244008004001210020021
:101FA0000084020800014400600020081080000145
:101FB0000500000A21000040084800200100010936
:101FC0000800200244008004001200000A002100E2
:101FD0000040288500104A8C148612033092C400F9
:101FE00000C030000048002001500000A080000127
:101FF000081004000600228000104000280061182C
:102000008661484A49229100F0FF00102C1E0D0203
:10201000004192270E10642B9300C458210E0041FA
:1020200097E3002196240F1C88C5620000922401CA
:1020300000204912008044220100F8010060A41031
:102040000080300C010008A51000200802070002E3
:10205000811008E40000411008211004812008418B
:1020600010288610468162F8611468A65F66815662
:10207000FEA71668E37F6C8176FCE31668A75F6EA7
:102080008120F84110208410428020F8411042A1A4
:10209000502824140A85424E1086204718638C214C
:1020A00084909F108240672E10080406020182600F
:1020B00010043300000000020200002010000000A5
:1020C0008400000080040000001100004000C300F4
:1020D0001000300C0400000101004000200010003E
:1020E00000040400008040000000300C000000C329
:1020F000000000000A0000001020000080008000A6
:102100000008000002C3000000380C00004000205E
:102110000000020080001000000082000000300C6F
:10212000200000C300800020000000020200000028
:10213000280000000024000000808000000010043F
:102140000000002100000010010000000900004014
:102150004000001010000004040000400100004096
:1021600004000010400000000202000040100000C7
:1021700000880000000009000000A00000000088A6
:102180000000000020020000008008000000002283
:10219000000000208000000002042F0080410000A9
:1021A00000100600000060100000000C010000801C
:1021B00030000000180200000061000000100C0058
:1021C0000000C2000000000C02000080300000008F
:1021D00000430000001804000084010000601000AB
:1021E000001006000080210000000C0200004030BA
:1021F0000000000083000000100C000000610000DF
:1022000000180200008201000060100000100600AB
:102210000080210000401800000086000000300807
:10222000000000C1000000000C0100008030000030
:10223000000806000000601000000082010000207D
:102240000C000000C02000000008060000804100D3
:102250000000300400000803000080210000401846
:10226000000000860000003008000000C1000000EF
:102270002D0080000010001000800000020004000B
:10228000400020000000090000000204008000005F
:102290001000180080018003001C007800E001801D
:1022A00007091E0078F0E00100178F1E0074F1E8A6
:1022B0000241168F263844F128C247108F20FE04B1
:1022C0006108F24F108020FF040000F20F000000B0
:1022D000EF000000700C00000083000000101800E8
:1022E0000080810300001C380800C1818360101C3D
:1022F000381886C1818761181E711886E138866199
:1023000018C647188621FE046108F25F1080A0FFFE
:10231000070000FE3F0000C0EF0300007C3C00000F
:10232000C0830300001C300000C000020000040055
:10233000040002000090000000204000000028007F
:102340000100000000040000000010000000004038
:1023500000000000000100000000040000008000F8
:10236000000000100000000002000000400000001B
:102370000008000000420000C008020030421000C7
:102380008C108200238410040821040040080100FE
:1023900000420000001000000000020000004000A9
:1023A0000000000800000000010000002000000004
:1023B0000080000000000002000000000800000093
:1023C0000020000000008000000020040000082120
:1023D000000042080180104208208410420021843D
:1023E0001000082104004008010000420000000025
:1023F00000000000420021000040080900104008D1
:1024000040080800200142004044000210900010E3
:1024100000020206000010110800400220201040B7
:10242000000180020009004400020420880000101E
:1024300001110080082002004400800811000020E3
:102440004600001001880040020024100090008027
:1024500002402000041004820000C0300000000C84
:10246000030000C03000003092C4000000000000F3
:102470003092C4000000000000000000000023496A
:102480000C00000000000000000000000000000040
:1024900023490C00000000000023490C000000004C
:1024A000000C1086000300000000730800E10C001F
:1024B0000000000023490C000000000000000000A4
:1024C000007892E4010000000000000000007F1886
:1024D00086E10F0000000000000000000000000086
:1024E0008C14861203000000000000000000480C5D
:1024F000230100000000104A0020850000000010A9
:102500004A00208500000000100200008400000046
:102510000010020000840000000000000000000025
:1025200037000001020002000208010000842000C0
:102530000010208000020000450000802080000084
:10254000040400010088000008500000005400004E
:10255000000500022001000140018000100022005F
:10256000000208080040010040000801200000109F
:102570001400000028100000024040001010000865
:10258000800800000104004000A0001000000104C9
:102590000000008600000030200000800180000064
:1025A0000C00000160000000088200000410100010
:1025B00080004002001000400108000000070000F9
:1025C00040081000084000400010020008004008C9
:1025D00000010000212000000005040040009000E0
:1025E0001000A00004000804010002012080400047
:1025F000002011000000440800000280400040005C
:1026000000010208000002084000000500004180AF
:102610000000080210004001000211241FBECFEF8D
:10262000D4E0DEBFCDBF11E0A0E0B1E0E8EBFFE316
:1026300002C005900D92AE30B107D9F711E0AEE0BF
:10264000B1E001C01D92A83FB107E1F70E94001E52
:102650000C94DA1F0C940000EF92FF920F931F93DB
:10266000CF93DF939C01162FEA018091F00186172A
:1026700010F41091F001FE0165917491C9010E945E
:10268000201F24E230E0AC01429FC001439F900D27
:10269000529F900D1124DC0144E0B695A7954A9510
:1026A000E1F71196AA0FBB1FAC0FBD1FBC016F70E5
:1026B0007070FD01C591D49140E050E021E0E22E20
:1026C000F12C012F10E0C701062E02C0880F991FC0
:1026D0000A94E2F78C239D23892B59F0FA01EE0F1F
:1026E000FF1FEE5CFE4F80819181800F911F9183CF
:1026F0008083FA01EE0FFF1FEE5CFE4F20813181D7
:102700008091F00190E08217930760F480910501B9
:10271000833018F41182108205C08091F00190E09E
:10272000918380836F5F7F4F6031710531F4129622
:10273000FD01C591D49160E070E04F5F5F4F44327E
:10274000510509F0C0CFDF91CF911F910F91FF90FC
:10275000EF90089580E090E0FC01E25FFE4F108270
:10276000019684329105C1F78091000181508093D8
:10277000F101089580E587BD82E084BD85BD809329
:102780006E0080936F008DE08093810080E498E379
:10279000909389008093880083E08DBB85E08093CF
:1027A000690008956AE070E00E94341F6530710589
:1027B00014F465E070E080E29EE40E94341F7093A0
:1027C0008900609388000895AC0181E08093EA015C
:1027D00020E030E008C01092EF018091EF018823E3
:1027E000E1F32F5F3F4F24173507A8F30895DF92D9
:1027F000EF92FF920F931F93CF93DF93E82E20E089
:1028000030E0F901E658FE4F8081F901E256FE4FB3
:1028100080832F5F3F4F2432310599F7FF24F394D3
:10282000DD24D39453C0C0E0D0E0FE01EE0FFF1FC3
:10283000EE5CFE4F20813181DE01A658BE4F8C91A7
:1028400090E082179307A0F4808191813C91FE0172
:10285000E256FE4F2081831B91096E2D70E00E948D
:10286000201F260F20838081FE01EE53FE4F1FC0E4
:10287000208131818C9190E08E010E531E4F2817DC
:10288000390790F48C9120813181FE01E256FE4F90
:10289000408190E0821B930B6E2D70E00E94201F00
:1028A000461B4083808102C080819181F801808332
:1028B0002196C432D10509F0B8CFD092EA01109226
:1028C000EF018091EF018823E1F3F394EF1408F016
:1028D000AACF20E030E0F901EE0FFF1FEE5CFE4FC3
:1028E00080819181F901E658FE4F80832F5F3F4F31
:1028F0002432310581F7DF91CF911F910F91FF9025
:10290000EF90DF9008951F920F920FB60F9211244F
:102910008F9381E08093EF018F910F900FBE0F9006
:102920001F9018951F920F920FB60F9211248F933C
:102930009F938091F1018F5F8093F1019091F1015C
:1029400080910001981708F499C01092F1018091CC
:10295000EA01882309F492C01092EA018091C20131
:1029600080930E018091C30180930F018091C40177
:10297000809310018091C501809311018091C6015F
:10298000809312018091C701809313018091C80147
:10299000809314018091C901809315018091CA012F
:1029A000809316018091CB01809317018091CC0117
:1029B000809318018091CD01809319018091CE01FF
:1029C00080931A018091CF0180931B018091D001E7
:1029D00080931C018091D10180931D018091D201CF
:1029E00080931E018091D30180931F018091D401B7
:1029F000809320018091D501809321018091D6019F
:102A0000809322018091D701809323018091D80186
:102A1000809324018091D901809325018091DA016E
:102A2000809326018091DB01809327018091DC0156
:102A3000809328018091DD01809329018091DE013E
:102A400080932A018091DF0180932B018091E00126
:102A500080932C018091E10180932D018091E2010E
:102A600080932E018091E30180932F018091E401F6
:102A7000809330018091E501809331019091F101C3
:102A800080913101981710F05E9801C05E9A5F9AAC
:102A90005F989091F10180913001981710F05E9845
:102AA00001C05E9A5F9A5F989091F10180912F0129
:102AB000981710F05E9801C05E9A5F9A5F989091A7
:102AC000F10180912E01981710F05E9801C05E9A76
:102AD0005F9A5F989091F10180912801981710F00A
:102AE0005E9801C05E9A5F9A5F989091F101809123
:102AF0002901981710F05E9801C05E9A5F9A5F985E
:102B00009091F10180912A01981710F05E9801C010
:102B10005E9A5F9A5F989091F10180912B019817CE
:102B200010F05E9801C05E9A5F9A5F989091F101F3
:102B300080911F01981710F05E9801C05E9A5F9A0D
:102B40005F989091F10180912501981710F05E989F
:102B500001C05E9A5F9A5F989091F1018091240183
:102B6000981710F05E9801C05E9A5F9A5F989091F6
:102B7000F10180911E01981710F05E9801C05E9AD5
:102B80005F9A5F989091F10180911901981710F068
:102B90005E9801C05E9A5F9A5F989091F101809172
:102BA0001801981710F05E9801C05E9A5F9A5F98BE
:102BB0009091F10180911D01981710F05E9801C06D
:102BC0005E9A5F9A5F989091F10180912301981726
:102BD00010F05E9801C05E9A5F9A5F989091F10143
:102BE00080911101981710F05E9801C05E9A5F9A6B
:102BF0005F989091F10180911201981710F05E9802
:102C000001C05E9A5F9A5F989091F10180911301E3
:102C1000981710F05E9801C05E9A5F9A5F98909145
:102C2000F10180911C01981710F05E9801C05E9A26
:102C30005F9A5F989091F10180912201981710F0AE
:102C40005E9801C05E9A5F9A5F989091F1018091C1
:102C50001701981710F05E9801C05E9A5F9A5F980E
:102C60005E985F9A5F985E985F9A5F989091F10185
:102C700080911601981710F05E9801C05E9A5F9AD5
:102C80005F989091F10180911001981710F05E9873
:102C900001C05E9A5F9A5F989091F10180912D0139
:102CA000981710F05E9801C05E9A5F9A5F989091B5
:102CB000F10180912701981710F05E9801C05E9A8B
:102CC0005F9A5F989091F10180912101981710F01F
:102CD0005E9801C05E9A5F9A5F989091F101809131
:102CE0001B01981710F05E9801C05E9A5F9A5F987A
:102CF0009091F10180911501981710F05E9801C034
:102D00005E9A5F9A5F989091F10180910F019817F8
:102D100010F05E9801C05E9A5F9A5F989091F10101
:102D200080910E01981710F05E9801C05E9A5F9A2C
:102D30005F989091F10180911401981710F05E98BE
:102D400001C05E9A5F9A5F989091F10180911A019B
:102D5000981710F05E9801C05E9A5F9A5F98909104
:102D6000F10180912001981710F05E9801C05E9AE1
:102D70005F9A5F989091F10180912601981710F069
:102D80005E9801C05E9A5F9A5F989091F101809180
:102D90002C01981710F05E9801C05E9A5F9A5F98B8
:102DA0005E985F9A5F985E985F9A5F98299A2998D3
:102DB00028989F918F910F900FBE0F901F9018959C
:102DC0001F920F920FB60F9211248F938091EC01F6
:102DD0008F5F8093EC018091EC01823038F080911C
:102DE000ED018F5F8093ED011092EC018F910F90B8
:102DF0000FBE0F901F9018951F920F920FB60F9253
:102E000011248F938091EB018F5F8093EB01809170
:102E1000EB01823038F08091E8018F5F8093E80108
:102E20001092EB018F910F900FBE0F901F9018958D
:102E3000682F20E030E0482F50E0F901EE0FFF1F2F
:102E4000EE5CFE4F518340838091F001861728F499
:102E50008091F00190E0918380832F5F3F4F243277
:102E6000310559F70895CF92DF92EF92FF920F93B9
:102E70001F937C016B010E94101FCE18DF0808947D
:102E8000C11CD11CB6010E94201FE80EF91EB7011B
:102E900080E090E01F910F91FF90EF90DF90CF9036
:102EA00008952F923F924F925F926F927F928F92EE
:102EB0009F92AF92BF92CF92DF92EF92FF920F93C9
:102EC0001F93DF93CF93CDB7DEB728970FB6F89453
:102ED000DEBF0FBECDBF3C012B011A01B22EA02ECA
:102EE000EE828C2C9093040180930301681779077C
:102EF00018F01D821C8207C0861B970BBA010E9426
:102F0000201F7D836C836414750440F4C20186190C
:102F10009709B1010E94201F7D836C83809103017A
:102F2000909104010E94D21383E090E06CE370E082
:102F30000E9433177B018C0183E090E06CE370E02A
:102F40000E9433176B0181E090E06AE070E00E941C
:102F50003317962E81E090E064E070E00E94331712
:102F60006093050180E090E064E070E00E94331718
:102F70007B836A8321E0821631F41DE3E12EF12C7C
:102F800035E039830AC082E0881631F4B2E0EB2ED6
:102F9000F12C95E0998301C0998218861F828824BC
:102FA000992400E010E00DC680E090E0FC01EE0FF7
:102FB000FF1FEE5CFE4F118210822091F0010196FE
:102FC0008432910599F70894811C911CEA81FB8158
:102FD000E815F90520F40F5F1F4F8824992480918C
:102FE000E801882339F0809101018F5F809301010E
:102FF0001092E80180910101843011F410920101D6
:1030000080910101882311F48FEF11C0809101019B
:10301000813011F480E20BC080910101823011F403
:1030200080E105C080910101833019F481E0809333
:10303000F0018091ED01882381F01092ED018091E3
:1030400002018F5F8093020180910201853019F4A3
:1030500081E08093020138862F82F2E0EF16F104BE
:1030600041F48F8198856B2D42EE53E00E942C1322
:1030700024C023E0E216F10441F48F8198856B2D82
:1030800042EF50E00E942C1324C034E0E316F10418
:1030900041F48F8198856B2D4AE251E00E942C13F8
:1030A00024C085E0E816F10441F48F8198856B2DEA
:1030B00044EB51E00E942C1324C096E0E916F10481
:1030C00041F48F8198856B2D46ED51E00E942C13C1
:1030D00024C0E7E0EE16F10441F48F8198856B2D52
:1030E00040E652E00E942C1324C0F8E0EF16F104F1
:1030F00041F48F8198856B2D4AEE52E00E942C138B
:1031000024C029E0E216F10441F48F8198856B2DEB
:1031100048E553E00E942C1324C03AE0E316F10482
:1031200041F48F8198856B2D48E650E00E942C1366
:1031300024C08BE0E816F10441F48F8198856B2D53
:1031400040E755E00E942C1324C09CE0E916F104EE
:1031500041F48F8198856B2D46E955E00E942C1330
:1031600024C0EDE0EE16F10441F48F8198856B2DBB
:1031700044E656E00E942C1324C0FEE0EF16F10452
:1031800041F48F8198856B2D4AEC56E00E942C13F8
:1031900024C02FE0E216F10441F48F8198856B2D55
:1031A0004AE157E00E942C1324C030E1E316F104F9
:1031B00041F48F8198856B2D44E357E00E942C13D6
:1031C00024C081E1E816F10441F48F8198856B2DCC
:1031D00040E957E00E942C1324C092E1E916F10463
:1031E00041F48F8198856B2D4AE158E00E942C13A1
:1031F00024C0E3E1EE16F10441F48F8198856B2D34
:103200004AE458E00E942C1324C0F4E1EF16F104C4
:1032100041F48F8198856B2D48E658E00E942C136D
:1032200024C025E1E216F10441F48F8198856B2DCD
:1032300048EE58E00E942C1324C036E1E316F10456
:1032400041F48F8198856B2D44E859E00E942C133E
:1032500024C087E1E816F10441F48F8198856B2D35
:103260004CEB59E00E942C1324C098E1E916F104BC
:1032700041F48F8198856B2D4AE45AE00E942C130B
:1032800024C0E9E1EE16F10441F48F8198856B2D9D
:1032900044ED5CE00E942C1324C0FAE1EF16F10427
:1032A00041F48F8198856B2D48E45DE00E942C13DA
:1032B00024C02BE1E216F10441F48F8198856B2D37
:1032C0004AEF5DE00E942C1324C03CE1E316F104B8
:1032D00041F48F8198856B2D4AE95EE00E942C13A2
:1032E00024C08DE1E816F10441F48F8198856B2D9F
:1032F00044E25FE00E942C1324C09EE1E916F10431
:1033000041F48F8198856B2D44EE5FE00E942C1371
:1033100024C0EFE1EE16F10441F48F8198856B2D06
:103320004CEE50E10E942C1324C0F0E2EF16F104A1
:1033300041F48F8198856B2D4AE252E10E942C1353
:1033400024C021E2E216F10441F48F8198856B2DAF
:103350004EEE52E10E942C1324C032E2E316F10437
:1033600041F48F8198856B2D40E255E20E942C1329
:1033700024C083E2E816F10441F48F8198856B2D17
:1033800046E656E10E942C1324C094E2E916F104AB
:1033900041F48F8198856B2D4CE157E10E942C13ED
:1033A00024C0E5E2EE16F10441F48F8198856B2D7F
:1033B00040EC57E10E942C1324C0F6E2EF16F10412
:1033C00041F48F8198856B2D48EF57E10E942C13B3
:1033D00024C027E2E216F10441F48F8198856B2D19
:1033E0004EE158E10E942C1324C038E2E316F104A8
:1033F00041F48F8198856B2D46E558E10E942C138E
:1034000024C089E2E816F10441F48F8198856B2D80
:1034100046E659E10E942C1324C09AE2E916F10411
:1034200041F48F8198856B2D42EC59E10E942C1359
:1034300024C0EBE2EE16F10441F48F8198856B2DE8
:103440004AE35AE10E942C1324C0FCE2EF16F10477
:1034500041F48F8198856B2D48E55AE10E942C1329
:1034600024C02DE2E216F10441F48F8198856B2D82
:1034700044E85AE10E942C1324C03EE2E316F10412
:1034800041F48F8198856B2D48E45BE10E942C13F9
:1034900024C08FE2E816F10441F48F8198856B2DEA
:1034A0004EEF5BE10E942C1324C090E3E916F10477
:1034B00041F48F8198856B2D48EF5CE10E942C13BD
:1034C00024C0E1E3EE16F10441F48F8198856B2D61
:1034D00044E25DE10E942C1324C0F2E3EF16F104F4
:1034E00041F48F8198856B2D4CE95DE10E942C138E
:1034F00024C023E3E216F10441F48F8198856B2DFB
:1035000048EF5DE10E942C1324C034E3E316F1047C
:1035100041F48F8198856B2D40E75EE10E942C136A
:1035200024C085E3E816F10441F48F8198856B2D62
:1035300042E25FE10E942C1324C096E3E916F104F5
:1035400041F48F8198856B2D4CEC5FE10E942C1328
:1035500024C0E7E3EE16F10441F48F8198856B2DCA
:103560004CEF5FE10E942C1322C0F8E3EF16F10448
:1035700041F48F8198856B2D42EB50E20E942C1311
:1035800020C029E3E216F10441F48F8198856B2D68
:103590004AE951E20E942C131EC03AE3E316F104FB
:1035A00031F48F8198856B2D40E752E21DC08BE38B
:1035B000E816F10431F48F8198856B2D4EE353E2C8
:1035C00013C09CE3E916F10431F48F8198856B2DCB
:1035D00044EF53E209C0EDE3EE16F10439F48F81B4
:1035E00098856B2D48E754E10E942C130894811CA8
:1035F000911C2A813B812815390520F40F5F1F4F4C
:103600008824992480910201833011F082E001C066
:1036100084E03981381708F082C282E0C816D104EC
:1036200039F4C8016A2D42EE53E00E942C1321C0E8
:1036300093E0C916D10439F4C8016A2D4AE251E079
:103640000E942C1321C0E4E0CE16D10439F4C80145
:103650006A2D44EB51E00E942C1321C0F5E0CF16F7
:10366000D10439F4C8016A2D46ED51E00E942C13B3
:1036700021C026E0C216D10439F4C8016A2D40E603
:1036800052E00E942C1321C037E0C316D10439F454
:10369000C8016A2D4AEE52E00E942C1321C088E036
:1036A000C816D10439F4C8016A2D48E553E00E94D8
:1036B0002C1321C099E0C916D10439F4C8016A2D30
:1036C00048E650E00E942C1321C0EAE0CE16D10457
:1036D00039F4C8016A2D40E755E00E942C1321C03F
:1036E000FBE0CF16D10439F4C8016A2D46E955E054
:1036F0000E942C1321C02CE0C216D10439F4C80159
:103700006A2D44E656E00E942C1321C03DE0C3160A
:10371000D10439F4C8016A2D4AEC56E00E942C13FA
:1037200021C08EE0C816D10439F4C8016A2D4AE1DF
:1037300057E00E942C1321C09FE0C916D10439F430
:10374000C8016A2D44E357E00E942C1321C0E0E138
:10375000CE16D10439F4C8016A2D40E957E00E9421
:103760002C1321C0F1E1CF16D10439F4C8016A2D20
:1037700042EF50E00E942C1321C022E1C216D10476
:1037800039F4C8016A2D4AE158E00E942C1321C087
:1037900033E1C316D10439F4C8016A2D4AE458E074
:1037A0000E942C1321C084E1C816D10439F4C80149
:1037B0006A2D48E658E00E942C1321C095E1C916F5
:1037C000D10439F4C8016A2D48EE58E00E942C1348
:1037D00021C0E6E1CE16D10439F4C8016A2D44E8CF
:1037E00059E00E942C1321C0F7E1CF16D10439F41F
:1037F000C8016A2D4CEB59E00E942C1321C028E12E
:10380000C216D10439F4C8016A2D4AE45AE00E9474
:103810002C1321C039E1C316D10439F4C8016A2D33
:1038200044ED5CE00E942C1321C08AE1C816D1044B
:1038300039F4C8016A2D48E45DE00E942C1321C0D0
:103840009BE1C916D10439F4C8016A2D4AEF5DE045
:103850000E942C1321C0ECE1CE16D10439F4C8012A
:103860006A2D4AE95EE00E942C1321C0FDE1CF16CB
:10387000D10439F4C8016A2D44E25FE00E942C13A0
:1038800021C02EE1C216D10439F4C8016A2D44EEDC
:103890005FE00E942C1321C03FE1C316D10439F42C
:1038A000C8016A2D4CEE50E10E942C1321C080E229
:1038B000C816D10439F4C8016A2D4AE252E10E94C7
:1038C0002C1321C091E2C916D10439F4C8016A2D24
:1038D0004EEE52E10E942C1321C0E2E2CE16D1043A
:1038E00039F4C8016A2D40E255E20E942C1321C030
:1038F000F3E2CF16D10439F4C8016A2D46E656E149
:103900000E942C1321C024E2C216D10439F4C8014C
:103910006A2D4CE157E10E942C1321C035E2C316F9
:10392000D10439F4C8016A2D40EC57E10E942C13F0
:1039300021C086E2C816D10439F4C8016A2D48EFC7
:1039400057E10E942C1321C097E2C916D10439F423
:10395000C8016A2D4EE158E10E942C1321C0E8E213
:10396000CE16D10439F4C8016A2D46E558E10E940B
:103970002C1321C0F9E2CF16D10439F4C8016A2D05
:1039800046E659E10E942C1321C02AE2C216D10456
:1039900039F4C8016A2D42EC59E10E942C1321C070
:1039A0003BE2C316D10439F4C8016A2D4AE35AE157
:1039B0000E942C1321C08CE2C816D10439F4C8012E
:1039C0006A2D48E55AE10E942C1321C09DE2C916D8
:1039D000D10439F4C8016A2D44E85AE10E942C133D
:1039E00021C0EEE2CE16D10439F4C8016A2D48E4B4
:1039F0005BE10E942C1321C0FFE2CF16D10439F401
:103A0000C8016A2D4EEF5BE10E942C1321C020E318
:103A1000C216D10439F4C8016A2D48EF5CE10E9456
:103A20002C1321C031E3C316D10439F4C8016A2D27
:103A300044E25DE10E942C1321C082E3C816D10448
:103A400039F4C8016A2D4CE95DE10E942C1321C0B4
:103A500093E3C916D10439F4C8016A2D48EF5DE13A
:103A60000E942C1321C0E4E3CE16D10439F4C8011E
:103A70006A2D40E75EE10E942C1321C0F5E3CF16CA
:103A8000D10439F4C8016A2D42E25FE10E942C138F
:103A900021C026E3C216D10439F4C8016A2D4CECCA
:103AA0005FE10E942C131FC037E3C316D10439F421
:103AB000C8016A2D4CEF5FE10E942C131DC088E302
:103AC000C816D10439F4C8016A2D42EB50E20E94B5
:103AD0002C131BC099E3C916D10429F4C8016A2D1F
:103AE0004AE951E21AC0EAE3CE16D10429F4C8012A
:103AF0006A2D40E752E211C0FBE3CF16D10429F44E
:103B0000C8016A2D4EE353E208C02CE3C216D1046B
:103B100031F4C8016A2D44EF53E20E942C1346147D
:103B2000570448F48091030190910401EC81FD81D8
:103B30008E1B9F0B0BC06414750460F4809103010D
:103B4000909104012C813D81820F931F9093040179
:103B50008093030180910201823019F488E592E09C
:103B60000DC080910201833019F484EF91E006C00A
:103B70008091020180910301909104010E94D2136F
:103B800080910201823011F48DE014C08091020115
:103B9000833069F080910201843059F480930501EB
:103BA0008F8198856FEF40EE58E00E942C1381E0E2
:103BB00001C08E810E94F7138F81988501969887A6
:103BC0008F83EF81F885E215F30508F4EDC9289697
:103BD0000FB6F894DEBF0FBECDBFCF91DF911F911E
:103BE0000F91FF90EF90DF90CF90BF90AF909F909C
:103BF0008F907F906F905F904F903F902F9008959F
:103C0000BF92CF92DF92EF92FF920F931F93CF93C9
:103C1000DF938FEF84B982EF8AB98CE08BB980E5AE
:103C200087BD82E084BD85BD80936E0080936F0068
:103C30008DE08093810080E498E3909389008093E5
:103C4000880083E08DBB85E08093690078948FEFD6
:103C50008093F00180910301909104010E94D2139E
:103C6000E0E0F0E020E030E081919191280F391FF1
:103C700084E0E03CF807C1F7C9010E94151F81E00C
:103C80000E94F71381E090E06AE070E00E94331731
:103C9000663068F488EE93E06CED75E04DE650E038
:103CA0002FEF0FEFE5E0EE2ECC24C3940CC084E69A
:103CB00090E066E970E048E550E02FEF0FEFEE246A
:103CC000E39432E0C32E0E94511788EC90E06CEB35
:103CD00072E00E9433176B0181E090E065E070E0D4
:103CE0000E943317162F81E090E064E670E00E9496
:103CF00033179B01AC01B60180E090E0620F731FA7
:103D0000841F951F212F30E040E050E00E94471FA4
:103D1000790181E090E066E070E00E943317643042
:103D200090F4A7014C595F4F80E9C81681E0D8068E
:103D300028F47A0111E0C0E2D3E00CC07A0111E06E
:103D4000C4E6D0E007C08CE291E06CEB72E00E9428
:103D50003317EB0180E890E06FEF70E00E943317BB
:103D6000B62E81E090E060E870E00E943317062FE5
:103D7000C601BE01A7012B2DE12ECC24A4CFA0E0CB
:103D8000B0E0E5ECFEE10C94AB1FEC01A880B9803B
:103D9000CA80DB80A114B104C104D10441F484E2DF
:103DA000A82E89EDB82E8BE5C82E87E0D82EC60147
:103DB000B5012DE133EF41E050E00E94881F27EA72
:103DC00031E440E050E00E94691F7B018C01C60194
:103DD000B5012DE133EF41E050E00E94881FCA0198
:103DE000B9012CEE34EF4FEF5FEF0E94691F6E0DAB
:103DF0007F1D801F911F97FF04C06150704080405D
:103E00009048688379838A839B839B013F77C901AC
:103E1000CDB7DEB7EAE00C94C71F0E94BF1E08951D
:103E200089E091E00E94BF1E0895A0E0B0E0809379
:103E3000090190930A01A0930B01B0930C0108951E
:103E4000AA1BBB1B51E107C0AA1FBB1FA617B707C0
:103E500010F0A61BB70B881F991F5A95A9F78095DC
:103E60009095BC01CD01089597FB092E07260AD035
:103E700077FD04D0E5DF06D000201AF47095619537
:103E80007F4F0895F6F7909581959F4F0895A1E291
:103E90001A2EAA1BBB1BFD010DC0AA1FBB1FEE1FC4
:103EA000FF1FA217B307E407F50720F0A21BB30B0F
:103EB000E40BF50B661F771F881F991F1A9469F78B
:103EC00060957095809590959B01AC01BD01CF01E7
:103ED0000895629FD001739FF001829FE00DF11D54
:103EE000649FE00DF11D929FF00D839FF00D749F74
:103EF000F00D659FF00D9927729FB00DE11DF91F20
:103F0000639FB00DE11DF91FBD01CF01112408957C
:103F100097FB092E05260ED057FD04D0B8DF0AD036
:103F2000001C38F450954095309521953F4F4F4FE8
:103F30005F4F0895F6F790958095709561957F4F46
:103F40008F4F9F4F08952F923F924F925F926F92A3
:103F50007F928F929F92AF92BF92CF92DF92EF9219
:103F6000FF920F931F93CF93DF93CDB7DEB7CA1B9A
:103F7000DB0B0FB6F894DEBF0FBECDBF09942A88C5
:103F8000398848885F846E847D848C849B84AA846D
:103F9000B984C884DF80EE80FD800C811B81AA81FA
:103FA000B981CE0FD11D0FB6F894DEBF0FBECDBFC5
:083FB000ED010895F894FFCF24
:0E3FB800FF01012C01010100FF0100000000CB
:00000001FF
